:100000000C9406040C943E040C943E040C943E04A0
:100010000C943E040C943E040C943E040C943E0458
:100020000C943E040C943E040C9454280C94262901
:100030000C943E040C943E040C943E040C943E0438
:100040000C943E040C943E040C943E040C943E0428
:100050000C943E040C94D9230C943E040C943E045E
:100060000C943E040C943E040C943E040C943E0408
:100070000C943E040C943E040C943E040C943E04F8
:100080000C943E090C943E040C943E040C943E04E3
:100090000C943E040C943E040C943E040C943E04D8
:1000A0000C943E040C943E040C943E04F609D809CA
:1000B000DB09DE09E109E409E709EA09ED09F009CC
:1000C000F309530B590B5F0B640B690B6E0B730B2E
:1000D000780B7D0B820B870B8C0B910B970B3712D8
:1000E000371263126312CB12F613F613F613E912EA
:1000F0008213931393139329BA29B22ABA29B22AE5
:10010000062A292AB22A802A8F2A11100F0E0D0CD6
:100110000B0A091213141516180706050403020129
:10012000001B1C1D1E1F2019083231302F2E2D36AA
:100130003738393A3B171A343329282726253F40C8
:1001400041423C3D3E21352C2BFFFFFFFF24FF4465
:10015000454647232240804B8454915BA461BB6693
:10016000D569F26DFF80F33DFF43FF48FF4DFF521D
:10017000FF56FF5AFF5DFF60FF38FF33FF2EFF2A57
:10018000FF25FF23FF20FF13FF00FF35842C91255F
:10019000A41FBB1AD516F9EDFFE0FFDDFFB8FFB3D2
:1001A00087AA95A3A99DC199DCFFFFA7FFA5FF80A2
:1001B0001A803C805E808080A280C491E994FFA177
:1001C000FF0009002B004D006F009100C9E0B5E66B
:1001D000D9EBFFBD80C883D28DDA9FFFFFC9E4CE83
:1001E000FFD5FFDAFF781068105810481038102833
:1001F00010181004100420800070006000500040AF
:100200000030002000100000009000A000B000C0EE
:1002100000D800E000F000F010F02088109810A83E
:1002200010B810C810DC10F030F040E040604064BE
:10023000305430443034302430FFFF303C1C406CAC
:10024000205C204C203C202C201C20142C0A300444
:10025000407C208C209C20AC20BC20D620B430CA0E
:1002600030E030743084309430A430FFFF903CA4F0
:1002700040BC40D04000344454002445550025354E
:1002800056002636460027374700283848002939C7
:1002900049002A3A4A002B3B4B00A4948400A595C0
:1002A0008500A6968600A7978700A8988800A99938
:1002B0008900AA9A7900AB8A7A009B8B7B003C4C20
:1002C0005C002C4D5D002D3D5E002E3E4E002F3F0C
:1002D0004F00304050003141510032425200334310
:1002E0005300AC9C8C00AD9D8D00AE9E8E00AF9FE8
:1002F0008F00B0A09000B1A19100B2A28100B39292
:100300008200A393830134445401244555012535CB
:100310005601263646012737470128384801293932
:1003200049012A3A4A012B3B4B01A4948401A5952B
:100330008501A6968601A7978701A8988801A999A3
:100340008901AA9A7901AB8A7A019B8B7B013C4C8B
:100350005C012C4D5D012D3D5E012E3E4E012F3F77
:100360004F0130405001314151013242520133437B
:100370005301AC9C8C01AD9D8D01AE9E8E01AF9F53
:100380008F01B0A09001B1A19101B2A28101B392FD
:100390008201A3938329001E001F00200021002258
:1003A00000230024002500260027002D002E002A0F
:1003B000004A002B0014001A000800150017001C4A
:1003C0000018000C00120013002F00300031004B09
:1003D00000390004001600070009000A000B000D98
:1003E000000E000F0033003400280000004E00E132
:1003F0000000001D001B0006001900050011001080
:1004000000360037003800E50052004D00E000E201
:1004100000000000000000000000002C00000000B0
:1004200000115F105F500051004F0035003A003B53
:10043000003C003D003E003F0040004100420043C0
:1004400000440045004C00010001000100010001D2
:1004500000010001000100010046004700480001C2
:100460000001000100010001000100010001000184
:100470000001000100010001000100010001000174
:100480000000000100010000000100010001000166
:100490000001000100010001000100010001000154
:1004A0000001000100010000000000000000000049
:1004B0000001000000000001000100010001000136
:1004C0000001000100010001000100010001000124
:1004D0000001000100010001000100010001000114
:1004E0000001000100010001000100010001000104
:1004F00000010001000100010001000100010001F4
:1005000000010001000100010001000100010001E3
:1005100000010001000100000001000100000001D5
:1005200000010001000100010001000100010001C3
:1005300000010001000100010001000100000000B5
:1005400000000000000000010000000000010001A8
:10055000000100010001000100035F025F075F0668
:100560005F0B5F0A5F0100010001000100015F00F5
:100570005F01000100010001000100095F085F0D3B
:100580005F0C5F010001000100010001000100019A
:100590000001000100010001000100010001000153
:1005A0000001000100010001000100010000000144
:1005B0000001000000010001000100010001000134
:1005C0000001000100010001000100010001000123
:1005D0000001000000000000000000000001000019
:1005E0000000000100010001000100010000010104
:1005F00001010101010101020202020202020202E2
:1006000003030303030303030404040404040405B1
:100610000505050506060606060707070707080875
:100620000808090909090A0A0A0B0B0B0C0C0C0D26
:100630000D0D0E0E0E0F0F0F1010111111121213BF
:10064000131414151516161717181819191A1A1B3A
:100650001B1C1D1D1E1E1F20202122222324242599
:100660002626272829292A2B2C2D2D2E2F303132D2
:1006700032333435363738393A3B3C3D3E3F4041E2
:1006800042434445464748494A4C4D4E4F505153CA
:1006900054555658595A5B5D5E5F61626465666881
:1006A000696B6C6D6F7072737577787A7B7D7E8005
:1006B00082838587888A8C8E8F91939596989A9C51
:1006C0009EA0A2A3A5A7A9ABADAFB1B3B5B7BABC65
:1006D000BEC0C2C4C6C9CBCDCFD1D4D6D8DBDDDF36
:1006E000E2E4E7E9EBEEF0F3F5F8FAFDFF0E035A6A
:1006F00000650061006C003600350000000E035AF2
:1007000000650061006C0050004300000004030914
:100710000409023B00020100A0FA090400000103E1
:100720000101000921110100012240000705810398
:100730000800010904010001030000000921110162
:100740000001226D00070582032000011201000252
:1007500000000008455A6500010001020001050182
:100760000980A101850319012AB700150126B700E8
:10077000950175108100C0050C0901A101850419BE
:10078000012AA002150126A002950175108100C062
:1007900005010906A1018506050719E029E71500ED
:1007A00025019508750181020507190029EF15003B
:1007B000250195F0750181020508190129059505A6
:1007C00075019102950175039101C005010906A10A
:1007D00001050719E029E715002501950875018134
:1007E000029501750881010507190029FF150026EA
:1007F000FF00950675088100050819012905950572
:1008000075019102950175039101C00011241FBE6D
:10081000CFEFDAE0DEBFCDBF04B603FE18C0809193
:10082000830490918404A0918504B091860487305C
:10083000904BA740B04B59F410928304109284045B
:100840001092850410928604E0E0F8E3099511E027
:10085000A0E0B1E0EAE7F8E502C005900D92AC3AFD
:10086000B107D9F724E0ACEAB1E001C01D92A3388A
:10087000B207E1F70E9404200C943B2C0C9400007A
:100880000E9410050C94B31E0F931F93CF93DF9318
:10089000EC018B010E94350BC0318FE5D80729F0A0
:1008A000C131EFE5DE0749F01EC0F80182818823DF
:1008B00011F081E007C081E013C0F8018281882334
:1008C00071F082E00E945A1543E062E081E00E94EC
:1008D000E10F80E0DF91CF911F910F91089582E0A9
:1008E0000E947B15F1CFB801CE01DF91CF911F910E
:1008F0000F910C943F0FCF93C82F0E9457058C2F58
:10090000CF910C945F1081E00C94540580E00C941E
:10091000540583E290E00E94B82B823281F484E295
:1009200090E00E94B82B823051F485E290E00E9462
:10093000B82B91E0873109F090E0892F01C080E069
:10094000817008950E948904882319F00E94100A7A
:1009500002C00E94180A0E94200A0E943B050C94C3
:100960004E05CF93C82F811102C06FEF01C062E224
:1009700083E290E00E94D62BC11102C06FEF01C04C
:1009800062E084E290E00E94D62BC11102C06FEFBA
:1009900001C067E185E290E0CF910C94D62B0E94D4
:1009A000A20481E00E94B1040C94B51EDB01E82F83
:1009B000F0E0EE0FFF1FEB51FE4F94919C933196A8
:1009C000E4911196EC931197863131F480910501F1
:1009D00080FF02C098509C930895E82FF0E0EE0F3E
:1009E000FF1FEB5AFE4F8491DB018C933196E4910B
:1009F0001196EC930895853020F08FEFDA018C93F7
:100A000008956F30D0F7E62FF0E0BFE08B9FE00D48
:100A1000F11D1124E65FFE4FE491DA01EC93089595
:100A200060E084E70E94150E61E086E70E94150EE3
:100A300060E084E70E942D0E61E086E70C942D0EA5
:100A4000CF93DF931F92CDB7DEB7AE014F5F5F4FFD
:100A50000E94FB04E981F0E0E052FD4F1082109209
:100A6000B0011092B1011092B2011092B3010F9037
:100A7000DF91CF9108958091AF0181110EC081E087
:100A80008093AF018DE0809391009FB7F89423E0AD
:100A900020939900809398009FBF0895E1E7F0E0CC
:100AA00080818260808308958093B9010895809346
:100AB000B80108958091B4019091B501A091B6015B
:100AC000B091B70180739927AA27BB2724E0B69578
:100AD000A795979587952A95D1F782309105A1051D
:100AE000B10571F083309105A105B10569F040E0D1
:100AF0000197A105B10511F060E008C06FEF02C0D9
:100B00004FEF60E080E003C04FEF6FEF8FEF0C948A
:100B1000FF0C40E060E080E00C94FF0CE5E0F1E0C9
:100B20006581768182810E94330C482F872F0C9437
:100B3000FF0C5F926F927F928F929F92AF92BF92C3
:100B4000CF92DF92EF92FF920F931F93CF93DF9399
:100B50001F92CDB7DEB760910A0170910B018091B1
:100B600007010E94330CE62E972E882E60910C010F
:100B700070910D01809107010E94330C762E672E33
:100B8000582E85E0C82E81E0D82EF12CAA24A394FB
:100B9000B12C00E010E0AE014F5F5F4F602F8F2D52
:100BA0000E94FB0489818834C0F4F60125893689C6
:100BB000A501002E02C0440F551F0A94E2F724231A
:100BC000352390E0232B21F4282D4E2D692D03C0D1
:100BD000252D472D662D0E94B80C0F5F1F4F0F303B
:100BE0001105C9F6F394F2E0CF0ED11C85E0F8129E
:100BF000D0CF0F90DF91CF911F910F91FF90EF9089
:100C0000DF90CF90BF90AF909F908F907F906F902C
:100C10005F900895DF92EF92FF920F931F93CF930F
:100C2000DF9300D0CDB7DEB780910C0190E020912A
:100C30000A01821B91098038910514F09A9505C02C
:100C400081382FEF92070CF4939597FD03969595B5
:100C5000879595958795182F80910D0190E02091AB
:100C60000B01821B910997FD0396959587959595A4
:100C70008795082FD0900701E12CF12CBE016F5F02
:100C80007F4F8E2D0E94D6048A8182958F7060914D
:100C90000A01819F600D112470910B01809F700DDE
:100CA00011248D2D0E94330C462F282F672FC7014A
:100CB0000E94B80C8FEFE81AF80A28E4E216F10453
:100CC000E9F60F900F90DF91CF911F910F91FF9058
:100CD000EF90DF900895AF92BF92CF92DF92EF92A4
:100CE000FF920F931F93CF93DF93082F10910A0168
:100CF00080910C0190E0811B910997FD03969595D9
:100D0000879595958795D82FB0900B0180910D010F
:100D100090E08B19910997FD039695958795959588
:100D20008795C82F0E94822B68E470E00E94FA2AFF
:100D3000E12CF12C6C01DD24011103C0EC14FD0445
:100D4000C9F40E94822B8370A12E8D9FA00C1124C8
:100D50000E94822B83707B2D8C9F700D11246A2D35
:100D6000809107010E94330C462F282F672FC7015F
:100D70000E94B80C8FEFE81AF80A88E4E816F1042C
:100D8000D9F6DF91CF911F910F91FF90EF90DF90F7
:100D9000CF90BF90AF900895CF92DF92EF92FF92E5
:100DA0001F93CF93DF938091B4019091B501A091EF
:100DB000B601B091B7010090090104C0880F991FD6
:100DC000AA1FBB1F0A94D2F7182F80EEE82E82E0EC
:100DD000F82EC0E0D0E09FE3C92ED12CF70181911D
:100DE0007F01F4E08F9FC0011124CA32D10551F078
:100DF000C334D10539F02091050123FF09C0C43463
:100E0000D10531F48091040324E0829FC0011124B4
:100E10008034910520F4B601681B790B02C060E0B4
:100E200070E0610F7FEF809107010E94330C462F25
:100E3000282F672FCE010E94B80C2196C834D10507
:100E400069F6DF91CF911F91FF90EF90DF90CF90E7
:100E500008958F929F92AF92BF92CF92DF92EF92BE
:100E6000FF920F931F93CF93DF9300D0CDB7DEB7E0
:100E70008091B4019091B501A091B601B091B701F4
:100E80000090090104C0880F991FAA1FBB1F0A9474
:100E9000D2F7B82EA090070180EEE82E82E0F82E5F
:100EA00000E010E09FE3C92ED12CF70181917F0172
:100EB000F4E08F9FC00111240A32110551F0033470
:100EC000110539F02091050123FF09C004341105F3
:100ED00031F48091040324E0829FC0011124803406
:100EE000910520F44601881A990A02C0812C912CA0
:100EF000BE016F5F7F4F802F0E94D60469816B0D0A
:100F0000680D7FEF8A2D0E94330C462F282F672F04
:100F1000C8010E94B80C0F5F1F4F0834110529F655
:100F20000F900F90DF91CF911F910F91FF90EF9055
:100F3000DF90CF90BF90AF909F908F9008958F9249
:100F40009F92AF92BF92CF92DF92EF92FF920F9358
:100F50001F93CF93DF9300D0CDB7DEB78091B4015C
:100F60009091B501A091B601B091B701009009012F
:100F700004C0880F991FAA1FBB1F0A94D2F7B82E6E
:100F8000A090070180EEE82E82E0F82E00E010E04D
:100F90009FE3C92ED12CF70181917F01F4E08F9F4F
:100FA000C00111240A32110551F00334110539F042
:100FB0002091050123FF09C00434110531F480910B
:100FC000040324E0829FC00111248034910520F4A1
:100FD0004601881A990A02C0812C912CBE016F5FCC
:100FE0007F4F802F0E94D6046A816B0D680D7FEFC2
:100FF0008A2D0E94330C462F282F672FC8010E948C
:10100000B80C0F5F1F4F0834110529F60F900F9091
:10101000DF91CF911F910F91FF90EF90DF90CF90D4
:10102000BF90AF909F908F900895EF92FF920F9393
:101030001F93CF93DF93F82E0E94822B68E470E019
:101040000E94FA2AC0E0D0E08C011127F11003C001
:101050000C171D0789F40E94822BE82E0E94822B18
:101060006E2D782F809107010E94330C462F282F78
:10107000672FCE010E94B80C2196C834D10531F7F4
:10108000DF91CF911F910F91FF90EF900895EF9214
:10109000FF920F931F93CF93DF9300D0CDB7DEB7AE
:1010A0008091B4019091B501A091B601B091B701C2
:1010B0000090090104C0880F991FAA1FBB1F0A9442
:1010C000D2F7F82EE090070100E010E0BE016F5F5C
:1010D0007F4F802F0E94ED0469816F0D7A818E2DE4
:1010E0000E94330C462F282F672FC8010E94B80C8E
:1010F0000F5F1F4F0834110549F70F900F90DF91D4
:10110000CF911F910F91FF90EF900895EF92FF9272
:101110000F931F93CF93DF9300D0CDB7DEB78091AD
:10112000B4019091B501A091B601B091B7010090C2
:10113000090104C0880F991FAA1FBB1F0A94D2F788
:10114000F82EE090070100E010E0BE016F5F7F4FD6
:10115000802F0E94ED0469816F0D67FD6095669593
:10116000669580910A01680F7A81769571588E2D67
:101170000E94330C462F282F672FC8010E94B80CFD
:101180000F5F1F4F0834110501F70F900F90DF918B
:10119000CF911F910F91FF90EF9008950F931F93A0
:1011A000CF93DF93082F809107010E94330CD62F35
:1011B000C72F182F0E3F41F4482F872FDF91CF9173
:1011C0001F910F910C94FF0C282F462F672F802F13
:1011D00090E00E94B80C043291F4212F4D2F6C2F17
:1011E0008BE290E00E94B80C212F4D2F6C2F84E4ED
:1011F00090E0DF91CF911F910F910C94B80CDF918B
:10120000CF911F910F910895809110018F3F51F060
:101210009091B80191FF06C060910E0170910F018D
:101220000E94CE0883E00E943A15882349F08091FD
:1012300019018F3F11F160911701709118011BC0C6
:1012400082E00E943A15882349F0809116018F3F71
:10125000A1F060911401709115010DC081E00E9410
:101260003A15882351F0809113018F3F31F060913E
:101270001101709112010C94CE0808951F920F92E3
:101280000FB60F9211240F931F932F933F934F93F9
:101290005F936F937F938F939F93AF93BF93CF93FE
:1012A000EF93FF938091AE01843120F48F5F8093A0
:1012B000AE01A2C08091B4019091B501A091B60198
:1012C000B091B7010196A11DB11D8093B401909317
:1012D000B501A093B601B093B7018091B001909190
:1012E000B101A091B201B091B3018F3F2FEF9207EE
:1012F000A207B20759F00196A11DB11D8093B0015C
:101300009093B101A093B201B093B301E0EEF2E08B
:1013100080818F3F11F08F5F8083319683E0E832C8
:10132000F807B1F7E0910801EF3F19F40E945A0560
:1013300063C08091B901882321F08091050185FD6A
:101340001EC0809106018823E1F020EB34E0829FEB
:10135000A001839F500D1124052E000C660B770B06
:1013600081E00091B0011091B1012091B201309162
:10137000B301401751076207730720F002C081E0F4
:1013800001C080E0C82FC17080FDE0E081E0909155
:1013900004019E1301C080E0E09304014E2F50E051
:1013A0004B30510518F5FA01EA5AFF4F0C94302BD7
:1013B0000E948E051DC00E9499051AC00E940A064F
:1013C00017C00E946B0614C00E94CC0611C00E9478
:1013D00029070EC00E949F070BC00E94150808C075
:1013E0000E94470805C00E94860802C00E94890525
:1013F000C11102C00E940409FF91EF91CF91BF91EA
:10140000AF919F918F917F916F915F914F913F919C
:101410002F911F910F910F900FBE0F901F90189555
:101420004FE150E067E270E085E091E00C94A82B7A
:101430004FE150E067E270E085E091E00C94C62B4C
:10144000CF93DF930E945F0E84E70E94680C86E7CB
:101450000E94680CC0E0D0E0C731D10529F480912A
:10146000050180FD04C007C0CA32D10521F061E04A
:10147000C334D10509F460E06170262F462F8C2F0C
:101480000E94190D2196C834D10531F760E084E738
:101490000E942D0E61E086E70E942D0EE0EEF2E044
:1014A0008FEF819393E0E832F907D9F7DF91CF917D
:1014B00008958091080190E001968B30910514F019
:1014C0008AE090E0809308010C94180A809108014A
:1014D00090E0019797FF02C080E090E08B3091058B
:1014E00014F08AE090E0809308010C94180A80912F
:1014F000090190E001968430910514F083E090E0BA
:10150000809309010C94180A8091090190E00197D9
:1015100097FF02C080E090E08430910514F083E0F2
:1015200090E0809309010C94180A8091070190E0E3
:1015300008968F3F910519F014F08FEF90E080939B
:1015400007010C94180A8091070190E0089797FF13
:1015500002C080E090E08F3F910519F014F08FEF0A
:1015600090E0809307010C94180A80910A0190E0A2
:1015700008968F3F910519F014F08FEF90E080935B
:101580000A010C94180A80910A0190E0089797FFCD
:1015900002C080E090E08F3F910519F014F08FEFCA
:1015A00090E080930A010C94180A80910B0190E05E
:1015B00008968F3F910519F014F08FEF90E080931B
:1015C0000B010C94180A80910B0190E0089797FF8B
:1015D00002C080E090E08F3F910519F014F08FEF8A
:1015E00090E080930B010C94180A80910C0190E01C
:1015F00008968F3F910519F014F08FEF90E08093DB
:101600000C010C94180A80910C0190E0089797FF48
:1016100002C080E090E08F3F910519F014F08FEF49
:1016200090E080930C010C94180A80910D0190E0D9
:1016300008968F3F910519F014F08FEF90E080939A
:101640000D010C94180A80910D0190E0089797FF06
:1016500002C080E090E08F3F910519F014F08FEF09
:1016600090E080930D010C94180A0F931F93CF9371
:10167000DF93EC018B01DB0112968C91129788238A
:1016800029F06C9111968C910E942005FE01FF5566
:10169000EE30F10508F050C0EF59FF4FD801129617
:1016A000CC910C94302BCC2309F447C00E94950AAE
:1016B0003CC0CC2309F441C00E94A30A36C0CC230D
:1016C000E1F10E94590A31C0CC23B9F10E94660AA7
:1016D0002CC0CC2391F10E94770A27C0CC2369F15A
:1016E0000E94840A22C0CC2341F10E94B50A1DC089
:1016F000CC2319F10E94C30A18C0CC23F1F00E9438
:10170000D50A13C0CC23C9F00E94E30A16C0CC232B
:10171000A1F00E94F50A09C0CC2379F00E94030BC6
:1017200004C0CC2351F00E94150BC0E006C0CC23AE
:1017300021F00E94230B01C0C1E08C2FDF91CF91DB
:101740001F910F910895EF92FF920F931F93CF93E4
:10175000DF938B01682F11110AC0442329F0E82F71
:10176000F0E0E351FA4F6491762F862F75C0212F58
:1017700030E0E82FF0E0442321F0E351FA4FE49108
:10178000F0E046E0049FC0011124CFEFD0E0BE019D
:101790000E94E62A4BEA4603C001479F900D1124A0
:1017A000800F911D800F911D982F990F890FAE0109
:1017B000421B530B4E9FD0014F9FB00D5E9FB00D4B
:1017C00011249B2F189FA0011124452F55278E010E
:1017D000041B150B0E9FA0010F9F500D1E9F500D57
:1017E00011247E01E81AF108E29E8001E39E100DAB
:1017F000F29E100D1124212F3327C21BD30BCE9F35
:101800009001CF9F300DDE9F300D112462307105A5
:10181000A9F048F46115710569F061307105C9F4EA
:101820008B2F752F0DC06430710581F058F0663034
:10183000710579F47E2F8B2F932F0DC0832F7B2F73
:101840009E2F09C08E2F7B2F952F05C08E2F732FB3
:1018500002C07E2F852F692FDF91CF911F910F91AD
:10186000FF90EF90089541E00E94A30B0895E8E4F3
:10187000F4E06083418324E630E042E050E0BF01C1
:10188000880F0C94160F0F931F93CF93DF93082F9D
:10189000000FEB0114E210934804E9E4F4E0DE01E8
:1018A0008D91819384E0E935F807D1F724E630E0A3
:1018B00041E150E068E474E0802F0E94160F105F51
:1018C0006096143B41F7DF91CF911F910F910895DE
:1018D000CF93DF93C82F4BE06DEF0E94370C40E0B1
:1018E0006AE08C2F0E94370C8FE39CE90197F1F797
:1018F00000C0000040E060E08C2F0E94370C40E008
:1019000061E08C2F0E94370C40E066E08C2F0E9433
:10191000370C40E06DEF8C2F0E94370CD0E040E098
:101920006D2F8C2F0E94370CDF5FD231C1F740E062
:101930006D2F8C2F0E94370CDF5FD432C1F740E04F
:101940006D2F8C2F0E94370CDF5FD43BC1F74BE02B
:101950006DEF8C2F0E94370C41E06AE08C2F0E94C3
:10196000370C40E06DEF8C2FDF91CF910C94370C4A
:10197000FF920F931F93CF93DF9300D000D0CDB78A
:10198000DEB78834910588F5122F042FF62EBC019E
:10199000660F771F660F771F6B587D4F44E050E04E
:1019A000CE0101960E94922B898183704A81282F53
:1019B00030E050E9859FC0011124885D9C4FFC01F7
:1019C000E40FF11DB497F0824B81FC01E40FF11D8F
:1019D000B49700834C81840F911DFC01B497108350
:1019E000F901E052FE4F81E080830F900F900F903D
:1019F0000F90DF91CF911F910F91FF900895FF926B
:101A00000F931F93CF93DF93182F062FF42EC0E070
:101A1000D0E02F2D402F612FCE010E94B80C2196CF
:101A2000C834D105B1F7DF91CF911F910F91FF908D
:101A300008955F926F927F928F929F92AF92BF9222
:101A4000CF92DF92EF92FF920F931F93CF93DF938A
:101A500000D000D0CDB7DEB7862E942E522E24E0D3
:101A6000829FC0011124BC016B587D4F44E050E0BF
:101A7000CE0101960E94922B2A8130E0C901849701
:101A8000FC0197FD379673E0F595E7957A95E1F7B8
:101A90004B8150E08A0104521109980117FF02C0DE
:101AA000295F3F4F63E0359527956A95E1F74C81B3
:101AB00050E05A0164E2A61AB1083501B7FE04C02D
:101AC0003A017DE1671A710843E0759467944A957D
:101AD000E1F758E0C52ED12CB6010E94FA2A7C010C
:101AE000C801B6010E94FA2A8C01C501B6010E9404
:101AF000FA2AFF274981FF24542F5370882081F050
:101B000062E1569FE00DF11D1124E454FE4F61E0A7
:101B100070E001C0660FEA94EAF75081652B10C0AF
:101B200072E1579FE00DF11D1124E454FE4F61E076
:101B300070E001C0660FEA94EAF760955081652372
:101B4000608333271127542F5370992089F062E165
:101B5000569F200D311D1124F901E454FE4F21E060
:101B600030E001C0220F0A95EAF73081232B11C023
:101B700072E1579F200D311D1124F901E454FE4FED
:101B800021E030E001C0220F0A95EAF7209530816C
:101B90002323208377249927942F93709301552032
:101BA000A1F052E1959F200D311D1124F901E4545B
:101BB000FE4F21E030E0B90102C0660F771F8A9521
:101BC000E2F7CB019081892B14C072E1979F200D21
:101BD000311D1124F901E454FE4F21E030E0B90138
:101BE00002C0660F771F8A95E2F7CB01809590813E
:101BF000892380834370E42FF0E0E654FE4F81E0B8
:101C000080830F900F900F900F90DF91CF911F91D5
:101C10000F91FF90EF90DF90CF90BF90AF909F908B
:101C20008F907F906F905F900895CF93DF93262FD2
:101C300030E0E901C052DE4F9881992351F090E9DC
:101C4000929FB001939F700D1124685D7C4F0E949C
:101C5000430C1882DF91CF910895DF92EF92FF92AB
:101C60000F931F93CF93DF93262F30E0A9014654A3
:101C70005E4F7A01FA01908191110AC0F70110823A
:101C8000DF91CF911F910F91FF90EF90DF9008951A
:101C9000D82EF2E16F9FE001112400E010E0F8017E
:101CA000EC0FFD1FE454FE4F4081602F8D2D0E94EC
:101CB000370C0F5F1F4F0231110589F7DFCF1092EC
:101CC000B9008CE08093B80008959F92AF92BF92C4
:101CD000CF92DF92EF92FF920F931F93CF93DF93F8
:101CE000B82EEB010E94B2236C01C431D10558F02B
:101CF000CF3F8FEFD80759F0CE0164E170E00E942A
:101D0000E62A7B0107C0EE24E394F12C03C025E012
:101D1000E22EF12C84E8A82E94EA992E1092BC00B1
:101D20009092BC000E94B2238C018091BC0087FD80
:101D300008C00E94B223801B910B8E159F05A8F34B
:101D40002AC08091B900887F883041F08091B90025
:101D5000887F803119F00FEF1FEF1FC0B092BB00DA
:101D6000A092BC000E94B2238C018091BC0087FD30
:101D700008C00E94B223801B910B8E159F05A8F30B
:101D80000AC08091B900887F883111F0803419F73A
:101D900000E010E00EC00EEF1FEFCF3F8FEFD8072F
:101DA00009F4BCCFC6010E94CA238C179D0708F412
:101DB000B5CFC801DF91CF911F910F91FF90EF90A8
:101DC000DF90CF90BF90AF909F9008950F931F9397
:101DD000CF93DF93EB018093BB0084E88093BC003A
:101DE0000E94B2238C018091BC0087FD0EC0CF3FC2
:101DF0008FEFD807C1F30E94B223801B910B8C1781
:101E00009D0788F38EEF9FEF0CC02091B900287FCB
:101E100081E090E0283211F480E090E09195819586
:101E20009109DF91CF911F910F910895CF92DF9289
:101E3000EF92FF920F931F93CF93DF936B018A0171
:101E40007901B9010E94650EE6010C0D1D1DC01738
:101E5000D10761F424E92093BC00DF91CF911F9159
:101E60000F91FF90EF90DF90CF90089597FDF2CF04
:101E7000B70189910E94E60EEACF81E0089581E0E2
:101E8000089508950C94410F1F93CF93DF9300D0D2
:101E900000D01F92CDB7DEB749835A836B83309150
:101EA000E30189819A81311114C0662359F02223FC
:101EB00049F00E944F16182F682F89819A810E943D
:101EC000F81503C00E942316182F69817A81812F8B
:101ED00004C00E944F1669817A810F900F900F9075
:101EE0000F900F90DF91CF911F910C94731DFC0107
:101EF000262F408151816281738184810C94440F2B
:101F000081E00895CF93DF93EC0160E00E94770FAA
:101F1000BE01DF91CF910C94420F8F929F92AF92AE
:101F2000BF92CF92DF92EF92FF920F931F936B01BC
:101F30007C0181E090E0A0E0B0E04C015D0104C0D4
:101F4000880C991CAA1CBB1C4A95D2F7AC01BD0198
:101F500004C0440F551F661F771F2A95D2F74829E2
:101F600059296A297B2904C0880F991FAA1FBB1F02
:101F70000A95D2F78A019B010C211D212E213F21B8
:101F8000401751076207730739F4BC01CD016C2972
:101F90007D298E299F290AC080959095A095B0959E
:101FA000BC01CD016C217D218E219F211F910F91BC
:101FB000FF90EF90DF90CF90BF90AF909F908F9069
:101FC00008950F93382F262F6091160270911702F3
:101FD0008091180290911902042F432F0E948D0FB7
:101FE0000F910C9414150C94CF040C944004089594
:101FF0000E9482140E94F70F2FEF84E39CE021508F
:1020000080409040E1F700C000000C94FF230F9344
:102010001F93CF93DF938C0161E00E94770FEC0157
:10202000B8010E9444048823F1F1B801CE010E9456
:10203000FD218823C1F1B801CE010E94112088231F
:1020400091F1B801CE010E945921882361F1F80174
:102050008281882309F1CB358DE5D807C1F050F492
:10206000C115FCE5DF0781F0CF3DDC45A9F40E94F6
:10207000861B19C0CC35EDE5DE0761F0CD35DD45B9
:1020800059F40E94C91A08C00E94F80F0CC00E949F
:10209000D21A02C00E94D51AC801DF91CF911F91B8
:1020A0000F910C943D0F80E0DF91CF911F910F9124
:1020B00008950C9483040E946E100C948604089575
:1020C00081E008950C9460100895CF93C82F0E946A
:1020D0007B048C2F0E946210CF9108950E94592298
:1020E0000C9465100E9459229091E201891721F009
:1020F0008093E2010C9465100895CF93DF93CDB7E0
:10210000DEB72B970FB6F894DEBF0FBECDBF4F835F
:10211000588769877A878B8761110E94151A9E01FB
:102120002F5F3F4F86E0F90111928A95E9F785E02C
:10213000FE013796D90101900D928A95E1F78981C8
:102140009A814C815D81452B31F09F3F31F491E0C4
:102150008F3F19F403C091E001C090E090FF09C0E7
:1021600049815A816B817C818D819E810E943619C3
:1021700005C0C9010E94800F8111F2CF2B960FB6C6
:10218000F894DEBF0FBECDBFDF91CF910895FC0163
:10219000808191810E9491160895CF93882309F43C
:1021A0009CC0C82F8238C1F40E94592281FD95C07D
:1021B00069E380912601909127010E9441230E94AA
:1021C000371A2FEF81EE94E0215080409040E1F7E4
:1021D00000C0000069E319C0833801F50E9459224C
:1021E00080FD7BC063E580912601909127010E94CC
:1021F00041230E94371A2FEF81EE94E02150804056
:102200009040E1F700C0000063E5809126019091C5
:1022100027010E944C23CF910C94371A8438C1F4C3
:102220000E94592282FD59C067E480912601909155
:1022300027010E9441230E94371A2FEF81EE94E07C
:10224000215080409040E1F700C0000067E4DDCFFE
:102250008CEF8C0F813AD0F46C2F809126019091F5
:1022600027010E94C122882349F06C2F809126010A
:10227000909127010E944C230E94371A6C2F809165
:102280002601909127010E944123C5CF80E28C0F47
:10229000883048F4C77081E001C0880FCA95EAF71A
:1022A0000E94F819B8CFEBE5EC0FE33040F4F0E012
:1022B000ED59FE4F808190E0CF910C947F22C85A57
:1022C000C73158F4EC2FF0E0EE0FFF1FEB5CFE4F30
:1022D00080819181CF910C949522CF91089588238C
:1022E00009F45BC0682F823879F40E94592281FF7B
:1022F00054C069E380912601909127010E944123F7
:102300000E94371A69E310C08338B1F40E94592241
:1023100080FF43C063E580912601909127010E94D0
:1023200041230E94371A63E580912601909127018D
:102330000E944C230C94371A843879F40E94592255
:1023400082FF2BC067E480912601909127010E94B3
:1023500041230E94371A67E4E7CF8CEF860F813A5A
:1023600018F380E2860F883048F4677081E001C07E
:10237000880F6A95EAF70E94FE19DCCF8BE5860F7D
:10238000833020F480E090E00C947F22685A67311B
:1023900020F480E090E00C94952208951F93CF9351
:1023A000DF93182FEB010E94CD10209741F08FE9A9
:1023B0009FE00197F1F700C000002197F6CF812F31
:1023C000DF91CF911F910C946F11893319F060E068
:1023D00070E002C060E570E00C94CE11882321F01B
:1023E0000E94F8190C94371A0895882321F00E944E
:1023F000FE190C94371A0895CF92DF92EF92FF9254
:102400000F931F93CF93DF937C01D62FC72FFC012F
:102410001281058102950F700E94EE198823B9F090
:102420001123A9F08C2F807F803421F080E28D0F62
:10243000883068F080915D0482FD09C082E00E94CE
:10244000971A0E94EE1991E0D82ED92601C0D12CFE
:10245000CC2EC2948FE0C8228C2D90E08C30910558
:1024600008F0C4C1FC01E159FF4F0C94302B8C2FB4
:10247000807FCF70882311F0C295C07F112399F01F
:10248000CC2309F49FC180E28D0F883010F0D11168
:1024900004C08C2F0E94F81903C08C2F0E94081AC8
:1024A0000E94371A8FC18D2F0E946F11CC2309F41F
:1024B0009DC180E28D0F883038F1DD2329F18C2F0A
:1024C0000E940E1A24C08C2F807FCF70803211F0B2
:1024D000C295C07FDD2319F0D130A1F13DC08091BC
:1024E0005D0482FF17C0112349F0CC2329F08C2F03
:1024F0000E94F8190E94371A80E065C180E00E94AE
:102500006F11CC2309F472C18C2F0E94FE190E9416
:10251000371A6CC1112371F0002341F0013031F4FE
:102520000E94181A8C2B0E94201A60C10E94181A4F
:102530008C2B1DC0002319F0013009F457C10E94F3
:102540002D1A25C0112321F0063008F04FC10EC00E
:10255000053008F04BC11BC0112361F0002331F09E
:10256000F701858180FF2EC18F7085838C2F0E949B
:10257000EE113CC1002359F0D93309F034C1FFEF0B
:1025800007EE13E0F15000401040E1F72AC18C2F14
:102590000E94F5112BC18C2F86958695837019F0BA
:1025A000813061F023C1112321F08D2F9C2F937076
:1025B00002C080E090E00E947F2220C1112321F020
:1025C0008D2F9C2F937002C080E090E00E94952296
:1025D00015C18C2F837009F047C011110BC12D2F2D
:1025E000229526952770220F220F6D2F6F70862F50
:1025F00090E0A0E0B0E0022E04C0880F991FAA1F4F
:10260000BB1F0A94D2F7D4FF10C04FE050E060E047
:1026100070E004C0440F551F661F771F2A95D2F73C
:10262000409550956095709503C040E050E0BA0128
:10263000C695C695C3708A019B01082B192B2A2BBE
:102640003B2BC901B801C23049F058F4C13019F030
:102650000E94EE14CFC00E94DC14CCC00E94001572
:10266000C9C00E94DA14C6C0112319F08C2F8170E2
:1026700001C08695882309F4BDC02D2F229526958B
:102680002770220F220F6D2F6F70862F90E0A0E031
:10269000B0E0022E04C0880F991FAA1FBB1F0A9426
:1026A000D2F7D4FF10C04FE050E060E070E004C00B
:1026B000440F551F661F771F2A95D2F740955095F6
:1026C0006095709503C040E050E0BA01C695C6958C
:1026D000C3708A019B01082B192B2A2B3B2BC901A4
:1026E000B801C23049F058F4C13019F00E94D31536
:1026F00081C00E94C1157EC00E94E5157BC00E946A
:10270000141578C0CF70112339F08C2F0E945A1500
:102710008D2F0E94EE116EC08D2F0E94F5118C2F0F
:102720000E947B1567C0D23F21F128F4D03F41F0D1
:10273000D13FC1F043C0D33F19F1D43F79F03EC03F
:10274000112341F0053008F051C08C2F8F710E9489
:10275000A0154CC0063008F049C0F7CF80915D0449
:1027600082FF18C0112339F08C2F8F710E945A15E7
:102770003DC01123C9F38C2F8F710E947B1536C089
:10278000112329F08C2F8F710E9445152FC00E94B4
:1027900020152CC0112349F0CF718C2F0E945A159F
:1027A00063E08C2F0E947C1A21C081E00E94971A5E
:1027B0000230E0F082E00E94971A18C0112331F035
:1027C000002391F28D2F0E94CD1010C0002399F2AA
:1027D000D93349F41FEF27EE33E011502040304049
:1027E000E1F700C000008D2F0E946F1188EF8C0D63
:1027F000843020F40E9459220E946510DD20C9F027
:102800000E94EA1980FD15C0F70112820E94E419A6
:102810000E945A15C7010E943A140E94E419DF91E0
:10282000CF911F910F91FF90EF90DF90CF900C947C
:102830007B15DF91CF911F910F91FF90EF90DF906B
:10284000CF9008950F931F93CF93DF93EC0168818E
:1028500079818A810E949C168C010E94F7150E9442
:10286000C814B801CE010E94FC11DF91CF911F91D5
:102870000F910895CF93DF93EC01988189812B818B
:102880003C81232B31F08F3F31F481E09F3F19F4DD
:1028900003C081E001C080E080FD1DC0CE010E9428
:1028A0000710811110C00E94EE198823A1F08A81BF
:1028B000882389F080915D0482FD0DC082E0DF9164
:1028C000CF910C94971ACE010E942214CE01DF9171
:1028D000CF910C94820FDF91CF91089580E090E02A
:1028E0000E947F2280E090E00E9495220E94151AAB
:1028F0000C94371A80912601909127010E9457234A
:102900000C946E140E94051A0C947A1492959F7080
:10291000963079F010F4925001C09A50923068F4D9
:10292000803F69F018F4883E40F409C0843F29F4E0
:1029300006C0883E20F0813F11F080E0089581E0DC
:102940000895FC01808191810E9491160E94861455
:102950000895CF93DF9300D000D01F92CDB7DEB79C
:102960000F900F900F900F900F90DF91CF910895DF
:10297000CF93DF9300D000D000D0CDB7DEB726963E
:102980000FB6F894DEBF0FBECDBFDF91CF91089593
:10299000089508950C94C9140C94CA140E94CC1480
:1029A00060931A0270931B0280931C0290931D0285
:1029B0000C946E140C94CE140F931F9300911A0272
:1029C00010911B0220911C0230911D02602B712B73
:1029D000822B932B1F910F910C94CE140F931F9366
:1029E00000911A0210911B0220911C0230911D02CD
:1029F00060237123822393231F910F910C94CE1493
:102A00000F931F9300911A0210911B0220911C0238
:102A100030911D0260277127822793271F910F9104
:102A20000C94CE140C94C9140E94121560931602D3
:102A30007093170280931802909319020C946E14ED
:102A400060E070E0CB010C941415611571058105EF
:102A5000910529F481E0442361F080E00895DC01D0
:102A6000CB0104C0B695A795979587954A95D2F75F
:102A700081700895482F609116027091170280911D
:102A80001802909119020C9425150F931F9341E0A1
:102A900050E060E070E08A019B0104C0000F111F4C
:102AA000221F331F8A95D2F7C901B8011F910F91D8
:102AB0000C9414150F931F9341E050E060E070E018
:102AC00004C0440F551F661F771F8A95D2F7809167
:102AD000160290911702A0911802B09119028A0172
:102AE0009B01082B192B2A2B3B2BC901B8011F91E5
:102AF0000F910C9414150F931F9341E050E060E088
:102B000070E004C0440F551F661F771F8A95D2F7E7
:102B1000409550956095709580911602909117029E
:102B2000A0911802B09119028A019B010823192370
:102B30002A233B23C901B8011F910F910C9414154E
:102B40000F931F9341E050E060E070E004C0440F39
:102B5000551F661F771F8A95D2F7809116029091B4
:102B60001702A0911802B09119028A019B0108274F
:102B700019272A273B27C901B8011F910F910C94EF
:102B800014150F931F9300911602109117022091B4
:102B9000180230911902602B712B822B932B1F91FD
:102BA0000F910C9414150F931F930091160210911E
:102BB0001702209118023091190260237123822399
:102BC00093231F910F910C9414150F931F93009151
:102BD00016021091170220911802309119026027F5
:102BE0007127822793271F910F910C941415089534
:102BF0002FE0929F800D1124E82FE695E695E6954B
:102C0000877051E001C0550F8A95EAF785E0E89F8B
:102C1000F0011124EC51FE4F20E030E070E04081E3
:102C2000CB01022E02C0969587950A94E2F7817037
:102C3000819584278523842781932F5F3F4F2530FB
:102C4000310569F708952FE0929F800D1124682FB8
:102C5000669566956695982F977085E0689FB00198
:102C6000112440E050E080E0FB01E40FF51FEC513F
:102C7000FE4F208130E0092E02C0369527950A9438
:102C8000E2F721703327042E01C0220F0A94EAF7DD
:102C9000822B4F5F5F4F4530510531F70895BF924A
:102CA000CF92DF92EF92FF920F931F93CF93DF9318
:102CB0008C01C0901602D0901702E0901802F0909C
:102CC000190280911A0290911B02A0911C02B091EE
:102CD0001D02C82AD92AEA2AFB2ACFE1D0E0D7016F
:102CE000C6010C2E04C0B695A795979587950A94B2
:102CF000D2F780FD04C0219790F7B12C07C0BC2EFD
:102D0000B8018C2F0E94861D0197A9F38B2DDF91AE
:102D1000CF911F910F91FF90EF90DF90CF90BF90D8
:102D20000895CF93DF93EC010E944F16BE010E94DD
:102D3000861DDF91CF9108951F93CF93DF93EB0111
:102D40009091E301992321F0CB010E94911613C0C9
:102D5000882349F0CB010E944F16182F682FCE010F
:102D60000E94F81504C0CB010E942316182FBE0143
:102D7000812F0E94861DDF91CF911F9108951F938F
:102D8000CF93DF93C0911E0216E080911F02C817F7
:102D900099F0D0E01C9FF0011D9FF00D1124E05E22
:102DA000FD4F4081518162817381848195810E94B0
:102DB000B8142196C770E9CFDF91CF911F91089584
:102DC0004091500250915102609152027091530211
:102DD00080915402909155020C94B814EF92FF9296
:102DE0000F931F93CF93DF938091550282958F703D
:102DF00009F065C080915202882309F460C0809177
:102E00001E02F0901F021091500200915102609139
:102E100053027091540291E01F3F09F090E0C0917D
:102E20002401D0912501292F96E0E92E8F1509F470
:102E300046C06115710521F00F3F21F030E003C05D
:102E400031E001C0322F90E030FD36C0E89EF00145
:102E5000E99EF00D1124DF01A05EBD4F11963C915B
:102E60001197301329C03C91311326C012963C9122
:102E70001297311121C013964D915C911497461B06
:102E8000570B4C175D07C0F4809155028F7080611D
:102E900080935502EB5DFD4F80818F708061808350
:102EA00080E592E00E943A14DF91CF911F910F913B
:102EB000FF90EF900C94BF1601968770B7CFDF910B
:102EC000CF911F910F91FF90EF9008959F92AF9235
:102ED000BF92CF92DF92EF92FF920F931F93CF9307
:102EE000DF93CDB7DEB761970FB6F894DEBF0FBEA4
:102EF000CDBF8C0185E0F801DE011D9601900D9299
:102F00008A95E1F7D8011296EC9090915002E091E9
:102F1000510220915302309154022115310531F0B4
:102F2000EF3F31F481E09F3F19F403C081E001C01D
:102F300080E0B82FB1709B2E80FD47C1D8014C9125
:102F400011965C9111971396AD90BC90149780E503
:102F5000C82E82E0D82EF0905202B501621B730B8E
:102F60002091240130912501FF2009F4D9C08091DE
:102F700055026217730708F095C0282F207F09F0CB
:102F800052C05E1313C0491311C0FE2CE1100EC0D5
:102F90008F708061809355020E94E016C6010E94E6
:102FA0003A1480915502F80185834DC1AB2831F068
:102FB0005F3F31F481E04F3F19F403C081E001C06D
:102FC00080E080FD03C081E08E2502C080E090E0BB
:102FD000F82FF170FF2E80FF1CC080911E022091FF
:102FE0001F0236E0821709F40BC190E0389FF00110
:102FF000399FF00D1124E05EFD4F6181561306C02C
:103000006081461303C06281E61203C00196877097
:10301000E9CFFE2CEE2009F416C1809155028160A3
:103020008093550254C05E1306C0491304C0E110DA
:1030300002C0F80199C0C8010E94A114882361F15F
:10304000EE2051F120915502822F82958F7090E0F1
:10305000029774F0809150029091510298878F836B
:103060001986BB86AA862C87CE0107960E943A1441
:1030700086E0F801A0E5B2E001900D928A95E1F7B3
:103080000E94EE160E94E0160AC05E1711F1C801F8
:103090000E94A11481112CC0C8010E943A14FF247F
:1030A000F394D1C0282F207F81F77A2DB98AA88A7E
:1030B0006E2D89890E94A91480E592E00E943A143D
:1030C00086E0D6011D928A95E9F70E94E016F12C60
:1030D000BAC04913DCCFE110DACFF8018583C8010B
:1030E0000E943A1486E0D6011D928A95E9F7ABC09A
:1030F000EE2091F220915502822F82958F7090E000
:1031000002970CF4B5CF80915002909151029A83AE
:1031100089831B82BD82AC822E83CE010196A6CF0D
:103120006217730708F044C0FE2CEE2009F4B4CFF8
:103130005E1330C049132EC02091550220FD21C0DE
:10314000822F82958F70482F50E041155105C9F0AC
:10315000F80125834F30510541F08F5F982F9295EC
:10316000907F822F8F70892B8583C8010E943A142B
:1031700086E0F801A0E5B2E001900D928A95E1F7B2
:103180003CC086E0F801A0E5B2E001900D928A957E
:10319000E1F759C0C8010E94A114811169CF809143
:1031A0005502816080935502C8010E943A144BC0B9
:1031B0007A2DB98AA88A6E2D89890E94A91486E081
:1031C000D6011D928A95E9F718C0EE2009F464CF64
:1031D000C8010E94A114F82E882309F45DCF86E06F
:1031E000F801A0E5B2E001900D928A95E1F780E543
:1031F00092E00E94C7100E94EE160E94E01623C0C3
:103200004D875E878D859E850E949116292F229578
:103210002F70223028F49F7039F0811105C00BC047
:10322000243028F49F7049F4805E883020F0C80173
:103230000E943A149F2CF92C06C0D80115969C9137
:10324000907F91F7F8CF8F2D61960FB6F894DEBF7F
:103250000FBECDBFDF91CF911F910F91FF90EF90E7
:10326000DF90CF90BF90AF909F9008951F93CF9322
:10327000DF93CDB7DEB72C970FB6F894DEBF0FBE45
:10328000CDBF4F83588769877A878B879C87CE010C
:1032900007960E9466178823D1F09F8188852A852A
:1032A0003B85232B31F08F3F31F481E09F3F19F4B0
:1032B00003C081E001C080E080FD47C04F81588598
:1032C00069857A858B859C850E94B8143EC086E00E
:1032D000FE013796DE01119601900D928A95E1F775
:1032E000FF81E8856A857B856115710531F0EF3FC7
:1032F00031F481E0FF3F19F403C081E001C080E0B8
:1033000080FD23C020911F0230E0C9010196877023
:10331000992740911E0250E084179507F1F1F98337
:10332000EA837D836C8396E0929FD001939FB00DDA
:103330001124A05EBD4FFE01319601900D929A9529
:10334000E1F780931F020E94BF1616E080911E02D3
:1033500090911F02891771F1189FC0011124805E9E
:103360009D4F0E946617882329F1E0911E021E9F3F
:10337000F0011124E05EFD4F408151816281738133
:10338000848195810E94B81480911E0290E001967C
:103390008770992780931E02D9CF0E9482141092C1
:1033A0001F0210921E02E0E5F2E086E0DF011D92AE
:1033B0008A95E9F72C960FB6F894DEBF0FBECDBF05
:1033C000DF91CF911F910895809176028595859523
:1033D0008595089580917602877008959091760280
:1033E000977081E009F480E0089580919902089532
:1033F00090919902892B80939902089580959091DC
:103400009902892380939902089510929902089550
:1034100090919802892B80939802089580959091BD
:103420009802892380939802089510929802089533
:1034300080917702089508950C941B1A0C941C1A1D
:1034400090915D0492FD08C090917702981721F049
:10345000809377020C941E1A089580917702882336
:1034600029F01092770280E00C941E1A0895CF93F1
:10347000DF93E0912601F0912701809199028083EA
:10348000E0912601F0912701908180919802892B8B
:10349000808380917702882381F0E0912601F0916A
:1034A00027019081892B80838091260190912701AB
:1034B0000E94AB2281110E942D1AC0912601D09149
:1034C000270140E250E066E572E0CE010E949B2BAE
:1034D000892B69F080E2FE01A6E5B2E001900D9231
:1034E0008A95E1F7CE01DF91CF910C946522DF91AF
:1034F000CF9108950C941B1A90915D0492FD10C019
:1035000098E0899F90011124262B209376020E9437
:103510005A15809176028595859585950C947A1A31
:103520000C945A151092760280E00C947A1A20912D
:1035300076028095822380937602982F977099F473
:1035400030E0482F082E000C550B2417350759F092
:1035500090915D0492FD07C08595859585950E94A3
:103560007B150C94921A089590915D0492FB22278A
:1035700020F9281769F080FB92F990935D048091FF
:103580005C0490915D040E94021B82E00C94971AE7
:10359000089580915D0482FB882780F991E0892756
:1035A0000C94B41A81E00C94B41A80E00C94B41A10
:1035B0006FEF7FEF80E090E00C94F42B80E090E0E0
:1035C0000E94C02B21E0893E9E4F09F020E0822F0F
:1035D000089582E090E00C94B82B83E090E00C9486
:1035E000B82BCF9384E090E00E94B82BC82F82E2E2
:1035F00090E00E94B82B2C2F30E0A901582BCA0173
:10360000CF910895CF93C92F682F84E090E00E9456
:10361000D62B6C2F82E290E0CF910C94D62BAB018D
:10362000BC018FE090E00C94E82BAB01BC0183E17E
:1036300090E00C94E82B60E070E0CB010C94151B3B
:1036400060E070E0CB010E940F1B0C941B1B69EE25
:103650007EEF80E090E00E94F42B60E082E090E05A
:103660000E94D62B60E083E090E00E94D62B10925F
:103670001A0210921B0210921C0210921D0260E0AE
:1036800084E090E00E94D62B60E082E290E00E940D
:10369000D62B60E085E090E00E94D62B60E086E0CB
:1036A00090E00E94D62B6FEF87E090E00E94D62B2F
:1036B00040E050E0BA0188E090E00E94E82B60E032
:1036C0008DE090E00E94D62B40E050E0BA0188E106
:1036D00090E00E94E82B60E087E190E00E94D62B0A
:1036E00040E050E0BA018CE190E00E94E82B60E0FD
:1036F00070E080E290E00E94F42B40E050E0BA01DC
:1037000088E190E00E94E82B0C94201B0C94271B6E
:10371000682F8EE090E00C94D62B0E94BE2360931D
:10372000A8027093A9028093AA029093AB026093BF
:10373000A4027093A5028093A6029093A702089515
:1037400085B7806885BF85B7806885BF089581E0AB
:1037500008950C94A71B08950C94AB1B0C94AB1B01
:103760000C94AE1B0C94AB1B0C94B21B0C94AB1BB7
:103770000E94A01B82E69EE10E944F220E94B61B7F
:103780000C94B41B0E94AC1B0C94AB1B0E947C1EBF
:103790000C9464100E94A9230E945D1F0E94C61B06
:1037A0000C94B01B5F926F927F928F929F92AF9218
:1037B000BF92CF92DF92EF92FF920F931F93CF931E
:1037C000DF93CDB7DEB72A970FB6F894DEBF0FBEF2
:1037D000CDBF0E94721FC82E81110E948D1B3AE935
:1037E000832E32E0932E00E010E0502E802F0E94B6
:1037F000A01E5C01F401619071904F01682679264A
:1038000061147104B1F40F5F1F4F0530110569F7A2
:103810008FEF89838A831B820E94B2238160782F75
:103820009D838C8349815A816B818D810E947D109B
:103830003AC08091AC0281FD0E94A91ED12CEE24D9
:10384000E394F12CC3018E219F21892B29F10E9441
:10385000A91B8823A9F0DE825F82AE20BF2081E011
:10386000AB2809F480E088870E94B2238160782F1A
:103870009A8789874E815F8168858A850E947D103D
:10388000000F111FF801E656FD4F80819181E82657
:10389000F926F182E08207C0D394EE0CFF1CFFE012
:1038A000DF12D0CFB0CF81E0C11001C080E02A96F6
:1038B0000FB6F894DEBF0FBECDBFDF91CF911F9141
:1038C0000F91FF90EF90DF90CF90BF90AF909F90BF
:1038D0008F907F906F905F9008950E94D21B0C9400
:1038E0007210CF93DF930E948B1DEC01811522E5AE
:1038F0009207E8F5811531E5930708F0B6C0883ED8
:10390000910528F5803E910508F0E9C0883A9105B7
:1039100070F4853A910508F07AC08130910509F478
:1039200073C008F4D9C0049708F0D9C0D5C08F3B44
:10393000910508F0D1C0C85AD0E0CC0FDD1FCA599C
:10394000DE4F0990D881C02DCE019464C9C0811585
:1039500040E5940708F069C0811550E4950708F028
:1039600060C09A9581159F4108F4B9C0B5C0811512
:1039700036E5930728F5811545E5940708F092C0D0
:10398000811554E5950708F087C0AC0143705527B1
:10399000282F26952695C115D34508F06CC081E0E7
:1039A00090E002C0880F991F4A95E2F740E2249FF9
:1039B00090011124EC01C22BD32BCE019C6890C046
:1039C00081152AE5920780F4811539E5930708F0FF
:1039D00072C0811548E5940708F47EC0D82FCC2723
:1039E000CE01806F906A7CC090568115904208F09D
:1039F00073C08D2F8F710E941F1EDD27D0628F71C3
:103A0000AE01582BCA016CC081E090E069C0C55A74
:103A1000D0E0CC56DE4F8881C82FD0E0CE01906434
:103A20005FC0DF70CE01906A5BC074E096958795A9
:103A30007A95E1F7282F23703C2F337081E090E0D6
:103A400002C0880F991F3A95E2F79C68AC01522B8F
:103A50009A019C2F9F709695969550E2959FE00154
:103A60001124C9018C2B9D2B3BC0D82FCC27CE0114
:103A7000816F906A35C081E090E002C0880F991F85
:103A80004A95E2F750E2259F90011124EC01C22BE8
:103A9000D32BCE019A6824C0D82FCC27CE01846FB7
:103AA000906A1EC00E941F1E8F7190E0D82FCC27F5
:103AB000CE01906215C08F700E941F1E94E0D695B3
:103AC000C7959A95E1F7CF70D0E0DC2FCC27D0696D
:103AD0009E01282BC90104C080E090E001C0CE0106
:103AE000DF91CF9108952BE4829FC0011124FC0146
:103AF0002FE0729FE00DF11D1124E60FF11DEE0F76
:103B0000FF1FEB56FC4F8591949108950E94731D01
:103B10000E94711C08958238910569F1B0F48133D7
:103B2000910509F46DC048F48932910509F463C028
:103B30008A32910509F469C008958533910509F425
:103B400055C089339105B9F00895833E910569F117
:103B500038F4803E9105B1F0823E910509F1089557
:103B6000863E9105A9F1873E9105B9F1843E910504
:103B700009F064C023C020915C0420FD4FC021FDEA
:103B80004DC0089580915C0480FD44C080915D0427
:103B900080FF44C080915C0484FD42C083EE4DC030
:103BA00080915C0482FF38C0F5CF80915C0482FD77
:103BB00033C080915D0480FD31C0ECCF80915D0405
:103BC00081FF32C080915C0484FD2AC087EE35C03D
:103BD00080915C0483FF26C0F5CF80915C0483FD57
:103BE00021C080915D0481FD1FC0ECCF80915C04F9
:103BF00085FD1CC01DC080915C0485FD19C016C0E8
:103C000080915C0486FD16C017C080915C0486FD1F
:103C100013C010C089E311C082EE0FC080EE0DC04A
:103C200080E00BC086EE09C084EE07C089E205C0C3
:103C300085E303C08AE201C081E390E0089590919A
:103C40005C0492FF0DC0282F2871283019F4877F5B
:103C5000846006C0282F2471243011F48B7F886083
:103C600093FF0DC0282F2871283119F4877E8461B5
:103C700006C0282F2471243111F48B7E8861209195
:103C80005D0420FF0DC0382F3871383019F4877F5C
:103C9000816006C0382F3171313011F48E7F886019
:103CA00021FF0DC0282F2871283119F4877E8161EA
:103CB00006C0282F2171213111F48E7E886194FD78
:103CC000877E089580E008950C94D81A0E94721F90
:103CD0008FE39CE90197F1F700C000000E94721F7A
:103CE00080E00E94A01E80FF04C00E94641E0C940D
:103CF000FF2308950C94661E0E94DE1A811102C0F3
:103D00000E94861B0E94E91A8093AC020E94F11A5D
:103D100090935D0480935C040E947A1E0E94ED1AC9
:103D2000682F70E080E090E00E94DA146091160243
:103D30007091170280911802909119020C9412153B
:103D4000E82FF0E0EE0FFF1FE859FB4F80819181D3
:103D50000895089580EA8A95F1F7089500C00895BE
:103D60000C94AA1E08950C94B21E0C94B21EF894E2
:103D7000E82FE295EF70F0E031A1282F2F7081E05D
:103D800090E001C0880F2A95EAF7982F9095932329
:103D900091A392A1892B82A3789408950F931F93E6
:103DA000CF93DF93C6EAD1E089918F3F11F00E9453
:103DB000B71E81E0CB3AD807B9F7C7E9D1E006EAE8
:103DC00011E089918F3F11F00E94B71E0C171D075B
:103DD000C1F7DF91CF911F910F910895BF92CF92BC
:103DE000DF92EF92FF920F931F93CF93DF938C019B
:103DF000C62FD0E0CE018A559E4F6C01FC01908108
:103E00009F3F09F450C0B62EF894E92FE295EF7069
:103E1000F0E081A19F7021E030E001C0220F9A956F
:103E2000EAF7822B81A382A12095282322A37894EC
:103E30000E94AE1EE7E9F1E046EA51E021E030E001
:103E4000E12CF12C61916F3F89F0A62FA295AF7004
:103E5000B0E090968C9190E06F7002C09595879538
:103E60006A95E2F780FD02C0C90102C080E090E0DF
:103E7000E82AF92A220F331F4E175F0719F7F601B8
:103E800080818F3F11F00E94B71E61E0E114F104C0
:103E900009F460E08B2D0E94B01ECC0FDD1FC00F17
:103EA000D11FF982E882DF91CF911F910F91FF908E
:103EB000EF90DF90CF90BF9008950E94CE1E8AE0D1
:103EC000E8E6F4E0DF01982F1D929A95E9F7EEE518
:103ED000F4E0DF011D928A95E9F785E00E94BD1F9D
:103EE0000C94F30FFF920F931F93CF93DF93CDB7F3
:103EF000DEB72A970FB6F894DEBF0FBECDBF8E0196
:103F00000F5F1F4F8AE0F80111928A95E9F7F12CB3
:103F10006F2DC8010E94EE1EF394F5E0FF12F8CF5A
:103F20004AE050E0B8018EE594E00E949B2BFF240C
:103F3000F394009709F4F12C892B41F08AE0F80101
:103F4000AEE5B4E001900D928A95E1F72F2D45E0A2
:103F500068E674E08EE594E00E94BE1F0E94F50FB3
:103F60008F2D2A960FB6F894DEBF0FBECDBFDF911E
:103F7000CF911F910F91FF9008950895FF920F9395
:103F80001F93CF93DF93F82E092F162FD72FC42F0F
:103F9000222349F081E08093AF020E94B2239093E4
:103FA000AE028093AD028091AF028823D9F0809158
:103FB000AD029091AE020E94CA23059798F0EF2DB2
:103FC000F02FA12FBD2F80E090E04C2F50E0841700
:103FD000950734F4219131912D933D930196F7CFBC
:103FE0001092AF02DF91CF911F910F91FF90089532
:103FF0000E94AC250E94CA1B0C94B8250E94BC25C7
:104000000E946D1C0C94D6250E949D230E9493252E
:104010000E94B81B0E94F81F0E94FE1F0E94C21B34
:10402000FBCFCF93DF93EC01FB018281882309F45E
:104030003CC1C430FDE5DF0760F4CB3F9CE5D90708
:1040400088F49E0122503C452431310508F02EC1F0
:1040500009C0C236EDE5DE0729F0C63AFDE5DF0707
:1040600009F024C10E94F11A90935D0480935C04CE
:10407000C1318CE5D80709F4C6C008F042C0C93088
:10408000ECE5DE0709F49BC000F5C5308CE5D807E8
:1040900009F485C078F4C330ECE5DE0709F478C094
:1040A00008F07AC0C230DC4509F0F5C080915C04AC
:1040B0008160EFC0C7309CE5D90709F478C008F0EB
:1040C0007AC080915C048061E4C0CD30FCE5DF07FC
:1040D00009F487C058F4CB309CE5D90709F479C0BE
:1040E00008F07BC080915C0488606FC0CF30FCE535
:1040F000DF0709F480C008F082C080915C04877FEC
:10410000C8C0CE3F9CE5D90709F471C000F5C531A0
:10411000FCE5DF0709F485C068F4C3319CE5D907E5
:1041200009F475C008F095C00E94821480915C0467
:104130008F77AFC0CC3FFCE5DF07A9F108F054C092
:10414000CB3FDC4509F0A7C080915D0440C0C23080
:10415000EDE5DE0709F489C058F4C1158DE5D807EF
:1041600009F45AC008F069C080915D0482602FC0D4
:10417000C236EDE5DE0709F47CC0C63AFDE5DF078F
:1041800009F481C0C330DD4509F085C080E06EC010
:1041900080915C0482607DC080915C0416C0809137
:1041A0005C04886076C080915D0482604FC080911D
:1041B0005C0480626EC080915C0480646AC00E946E
:1041C000821480915C04806864C0846062C08160F5
:1041D0003DC080915C048E7F5CC080915C048D7FCB
:1041E00058C080915C0416C080915D0418C0809115
:1041F0005D048D7F2BC080915C048F7E4AC08091CE
:104200005C048F7D46C080915C048F7B42C08091AE
:104210005C04877F8B7F3DC080915D048D7F8E7FA6
:1042200015C080915C0482FB222720F991E092273F
:1042300090FB82F990FB83F92CC080915D04982F4C
:10424000909591708E7F892B90FB81F980935D040E
:1042500022C00E94821480915C0487FB222720F9EF
:1042600091E0922790FB87F914C081E00E94881B9F
:1042700012C080915C0484FB222720F991E09227F0
:1042800090FB84F906C080915C04982F909590FB78
:1042900080F980935C0480915C0490915D040E949D
:1042A000021B0E94821480E001C081E0DF91CF9167
:1042B0000895CF93DF9386319C4541F5EB010E9431
:1042C000F519982F8A8120912601309127018823A2
:1042D00079F09A7A81E009F480E08093B00291113C
:1042E00002C069E201C065E3C9010E9441230AC01E
:1042F0008091B002811102C069E201C065E3C90189
:104300000E944C230E94371A80E001C081E0DF91B7
:10431000CF9108950F931F93CF93DF93C42FD22F84
:10432000FC0182818823C9F04093B3020E94B2232A
:104330009093B2028093B10280E28C0F883008F033
:1043400057C0C77081E001C0880FCA95EAF7DF91B6
:10435000CF911F910F910C94EE118091B3024813ED
:1043600030C08091B1029091B2020E94CA23883C71
:10437000910538F510E21D0FCD17B9F080E28C0FD2
:10438000883040F4C77081E001C0880FCA95EAF711
:104390000E94F511183028F581E09D2F977001C01B
:1043A000880F9A95EAF70E94EE11802F0E94E5117E
:1043B0001830F0F4D77081E001C0880FDA95EAF781
:1043C0000AC080E28C0F883098F4C77081E001C089
:1043D000880FCA95EAF7DF91CF911F910F910C9446
:1043E000F511802FDF91CF911F910F910C94E51162
:1043F000DF91CF911F910F9108950F939C01CB01F5
:10440000243F4CE5340731F188F4293DFCE53F07B2
:10441000D9F02A3D4CE5340779F1283D3C45A9F512
:1044200006E221EE41EE68ED7CE52BC0263FFCE57F
:104430003F07E1F0A8F0273F3C4539F507E225EEBC
:1044400046EE67EF7CE51DC007E225EE45EE69ED1F
:104450007CE517C006E221EE40EE64EF7CE511C07A
:1044600007E225EE44EE65EF7CE50BC006E221EEA7
:1044700042EE66EF7CE505C008E221E045EE6AED1C
:104480007CE50E948A2180E008C0FC0182818823AB
:1044900019F01092B30201C081E00F91089590933A
:1044A000AD018093AC0108959093B9028093B80256
:1044B0000895E091B802F091B902309721F001908F
:1044C000F081E02D099480E00895E091B802F09128
:1044D000B902309799F020913401222359F02091AC
:1044E0005C0427FF07C0DC012C9111962C931197D7
:1044F00026E02C930280F381E02D09940895209109
:10450000B6023091B7022817390771F09093B702BD
:104510008093B602E091B802F091B902309721F091
:104520000680F781E02D099408952091B40230911E
:10453000B5022817390771F09093B5028093B40241
:10454000E091B802F091B902309721F00084F18532
:10455000E02D09940895FC0132968091340188235E
:1045600031F080915C0487FF02C09EE101C096E0BB
:1045700080E0915028F021912223D9F38F5FF9CF69
:104580000895662351F1209134012223E9F020910E
:104590005C0427FF19C0462F4695469546954E3137
:1045A000E0F4677021E030E002C0220F331F6A950B
:1045B000E2F7FC01E40FF11D828190E0282339230A
:1045C00081E0232B69F409C0FC0132960896219101
:1045D000621729F0E817F907D1F780E0089581E024
:1045E00008959C01FC0132969FEF80E041914617AF
:1045F00089F09F3F19F4411101C0982F8F5F8630D9
:10460000A9F79F3F39F0F901E90FF11D97FDFA95E0
:104610006283089508959C012A5F3F4FFC01428107
:10462000461301C01282019682179307B9F70895C5
:10463000262F2695269526952E3168F4FC01E20F4B
:10464000F11D677021E030E001C0220F6A95EAF7A2
:104650008281282B22830895262F2695269526953C
:104660002E3170F4FC01E20FF11D677021E030E0A3
:1046700001C0220F6A95EAF72095828128232283C0
:10468000089520913401222329F020915C0427FD14
:104690000C9418230C94F12220913401222329F048
:1046A00020915C0427FD0C942C230C940B23209167
:1046B0003401FC013296222331F080915C0487FFA3
:1046C00002C08EE101C086E0DF011D928A95E9F704
:1046D000089508950C94692383E08093BA020C94A2
:1046E0006A23811102C081E001C082E08093BA0296
:1046F0000C946A230C94712381E08093BA020C9489
:104700006A230C947C2308950C9483230C948323B4
:10471000CF930E9486230E94721F0E948423C0E0D0
:104720008C2F0E94A01E892B29F4CF5FC530C1F7C2
:1047300080E001C081E0CF910895089580917A04CE
:10474000843011F00C94591008950E9482140C9436
:104750005B1082E084BD93E095BD9AEF97BD809396
:104760006E0008952FB7F8948091720490917304AD
:10477000A0917404B09175042FBF08952FB7F894D9
:104780006091720470917304809174049091750427
:104790002FBF08959C014FB7F894809172049091B7
:1047A0007304A0917404B09175044FBF821B930BE6
:1047B000089578941F920F920FB60F9211248F9341
:1047C0009F93AF93BF938091720490917304A091D3
:1047D0007404B09175040196A11DB11D80937204FB
:1047E00090937304A0937404B0937504BF91AF9138
:1047F0009F918F910F900FBE0F901F90189581E0A1
:104800008093E00080E28093D8001092C9008FE18D
:104810009EE40197F1F700C0000087E090EBDC0117
:104820008093830490938404A0938504B0938604BA
:104830009CE088E10FB6F894A895809360000FBEC5
:1048400090936000FFCF8091DE0208950895CF938A
:10485000DF9320913401222339F020915C0427FF5B
:1048600003C060E222E002C068E021E02093E9009A
:104870002FEF3091E800215035FD06C035ED3A9517
:10488000F1F700002111F5CF2091E80025FF1DC0B0
:10489000EC0180913401811105C040E050E068E0F6
:1048A00070E003C070E040E050E0CE010E94482676
:1048B0008091E8008E778093E80080E2FE01AEEB05
:1048C000B2E001900D928A95E1F7DF91CF910895C2
:1048D0008093BB027093BD026093BC0280917A0406
:1048E000843001F582E08093E9008FEF9091E80039
:1048F000815095FD06C095ED9A95F1F70000811164
:10490000F5CF8091E80085FF0DC040E050E063E006
:1049100070E08BEB92E00E9448268091E8008E7751
:104920008093E8000895BC0184E00C946824BC01E5
:1049300083E00C946824089580917904811109C062
:104940000E94D9270E9436288091E20084608093DB
:10495000E20008951092790408950C9481236091E7
:10496000760481E0611101C080E00C946C23909189
:104970007A0481E0943009F080E0609176040C9430
:10498000712342E061EC81E00E94522742E261EC37
:1049900082E00E94522790917A0481E0943009F0DD
:1049A00080E0609176040C947A2380917C048330BB
:1049B00009F461C030F4813071F0823009F49AC09A
:1049C00008958A3009F486C08B3009F46CC08930B0
:1049D00009F0A8C020C080917B04813A09F0A2C0F0
:1049E0008091E800877F8093E80080917F04909118
:1049F0008004892B21F460E28EEB92E003C060E03A
:104A000080E090E070E00E9493268091E8008B7730
:104A10008093E800089580917B04813209F082C080
:104A200080917F0490918004029708F07BC0809170
:104A3000E800877F8093E8008091E80082FD05C050
:104A400080917A048111F8CF6DC02091F30080919C
:104A5000F20090E0922B029731F48091F1008130C6
:104A600011F0863021F48091F1008093DE02809174
:104A7000E8008B7753C080917B04813A09F052C0E3
:104A800080917F0490918004892B09F04BC0809124
:104A9000E800877F8093E8008091E80080FFFCCFEA
:104AA0008091340136C080917B048132D9F58091A8
:104AB0007F0490918004892BA9F58091E800877F7D
:104AC0008093E8000E94872780917D0480933401C1
:104AD0000C94821480917B04813221F58091E8004E
:104AE000877F8093E8000E94872780917E048093CF
:104AF000DF02089580917B04813AA1F48091E8005F
:104B0000877F8093E8008091E80080FFFCCF809150
:104B1000DF028093F1008091E8008E778093E800B7
:104B20000C948727089584B7877F84BF0FB6F894C5
:104B3000A895809160008861809360001092600069
:104B40000FBE90E080E80FB6F894809361009093D8
:104B500061000FBE0C947C230E94D9270E94362846
:104B6000E2EEF0E080818460808378940C94CB2A1C
:104B700088E291E00C94542280917A048530A9F463
:104B800080917A04853079F40E949E238091780484
:104B90008823B1F30E948823882391F30E94322650
:104BA0000E948214EDCF0C94A523089508950C94CF
:104BB000D925292F332723303105C9F060F421305E
:104BC000310581F02230310509F044C08BE390E0DB
:104BD00021E137E043C021323105E1F022323105D5
:104BE00049F138C082E190E02CE437E037C09927E2
:104BF0008130910549F028F0029761F5EDEEF6E07D
:104C000005C0EDE0F7E002C0EDEFF6E0849190E042
:104C10009F0124C06115710541F061307105D1F427
:104C200089E090E02CE337E019C089E090E023E2CE
:104C300037E014C06115710541F06130710551F420
:104C40008DE690E02EE537E009C080E490E02BECA3
:104C500037E004C080E090E020E030E0FA013183EA
:104C60002083089580E189BD82E189BD09B400FEF9
:104C7000FDCF8091D8008F7D8093D8008091E00097
:104C800082608093E0008091E00081FDFCCF089578
:104C9000CF92DF92EF92FF920F931F93CF93DF9308
:104CA000EC018B017A010E94A627811133C0E11427
:104CB000F10439F0F70180819181081B190BC80FAD
:104CC000D91FC12CD12C0115110519F18091E800D3
:104CD00085FD16C08091E8008E778093E800E1148E
:104CE000F10449F0F70180819181C80ED91ED1826B
:104CF000C08285E00FC00E94A627882321F30AC046
:104D000089918093F10001501109FFEFCF1ADF0A5A
:104D1000DACF80E0DF91CF911F910F91FF90EF905C
:104D2000DF90CF900895209181043091820426175E
:104D3000370748F06115710539F42091E8002E77A6
:104D40002093E80001C0B901FC0120E06115710564
:104D500079F180917A048823F1F18530F1F1809125
:104D6000E80083FD3CC08091E80082FD2EC0809168
:104D7000E80080FFEBCF2091F3008091F20090E0FB
:104D8000922B6115710551F08830910538F421910D
:104D90002093F100615071090196F3CF21E008974B
:104DA00009F020E08091E8008E778093E800CECF74
:104DB0002111CFCF0AC080917A04882361F0853019
:104DC00061F08091E80083FD0AC08091E80082FFD5
:104DD000F2CF80E0089582E0089583E0089581E0B5
:104DE000089520918104309182042617370748F0F6
:104DF0006115710539F42091E8002E772093E800C1
:104E000001C0B901FC0120E06115710591F18091AB
:104E10007A04882309F440C0853009F43FC08091AA
:104E2000E80083FD3DC08091E80082FD2FC08091A5
:104E3000E80080FFE9CF2091F3008091F20090E03C
:104E4000922B6115710559F08830910540F4249139
:104E50002093F1003196615071090196F2CF21E063
:104E6000089709F020E08091E8008E778093E800B1
:104E7000CBCF2111CCCF0AC080917A04882361F076
:104E8000853061F08091E80083FD0AC08091E800E0
:104E900082FFF2CF80E0089582E0089583E00895D4
:104EA00081E00895982F973068F59093E90098175E
:104EB00039F07091EC002091ED005091F00003C0AA
:104EC000242F762F50E021FD02C09F5FECCF309160
:104ED000EB003E7F3093EB003091ED003D7F30934F
:104EE000ED003091EB0031603093EB007093EC00FB
:104EF0002093ED005093F0002091EE0027FDE5CFC8
:104F000080E008958F708093E90081E0089580919A
:104F10007B0487FF11C08091E80082FD05C080916D
:104F20007A048111F8CF11C08091E8008B770BC013
:104F300080917A04882349F08091E80080FFF8CFBF
:104F40008091E8008E778093E80008952091E40036
:104F50003091E50095E64091EC00842F817040FF90
:104F600023C08091E80080FD1DC080917A048823D1
:104F700099F0853099F08091EB0085FD11C040914A
:104F8000E4005091E5002417350729F3915011F002
:104F90009A01E1CF84E0089582E0089583E00895C6
:104FA00081E0089580E008954091E80042FFDDCF60
:104FB00008950E9447280E944F28E0EEF0E080818B
:104FC00081608083E8EDF0E080818F77808319BC79
:104FD000A7EDB0E08C918E7F8C9380818F7E808353
:104FE0001092790408950F931F93CF93DF930E943B
:104FF00047280E944F28C8EDD0E088818F778883AA
:1050000088818068888388818F7D888319BC10920D
:105010007A0410927604109278041092770400EECD
:1050200010E0F80180818B7F808388818160888394
:1050300042E060E080E00E945227E1EEF0E08081F3
:105040008E7F8083E2EEF0E08081816080838081CA
:1050500088608083F80180818E7F80838881806171
:105060008883DF91CF911F910F910895E8EDF0E0D3
:1050700080818F7E8083E7EDF0E080818160808396
:1050800084E082BF81E0809379040C94F327E8EDFB
:10509000F0E080818E7F80831092E200089510926C
:1050A000DA001092E10008951F920F920FB60F924E
:1050B00011242F933F934F935F936F937F938F931D
:1050C0009F93AF93BF93EF93FF938091E10082FF93
:1050D0000BC08091E20082FF07C08091E1008B7FCE
:1050E0008093E1000E94CA2A8091DA0080FF1FC0ED
:1050F0008091D80080FF1BC08091DA008E7F809362
:10510000DA008091D90080FF0DC080E189BD82E185
:1051100089BD09B400FEFDCF81E080937A040E942E
:105120009C2405C019BC10927A040E94AA24809184
:10513000E10080FF19C08091E20080FF15C08091DE
:10514000E2008E7F8093E2008091E2008061809394
:10515000E2008091D80080628093D80019BC85E07D
:1051600080937A040E94AF248091E10084FF30C0D4
:105170008091E20084FF2CC080E189BD82E189BD7D
:1051800009B400FEFDCF8091D8008F7D8093D800B8
:105190008091E1008F7E8093E1008091E2008F7E1C
:1051A0008093E2008091E20081608093E200809130
:1051B0007604882311F084E007C08091E30087FD26
:1051C00002C081E001C083E080937A040E94B7248A
:1051D0008091E10083FF29C08091E20083FF25C018
:1051E0008091E100877F8093E10082E080937A04E0
:1051F000109276048091E1008E7F8093E10080918F
:10520000E2008E7F8093E2008091E20080618093D3
:10521000E20042E060E080E00E9452278091F000CE
:1052200088608093F0000E94AD24FF91EF91BF91C0
:10523000AF919F918F917F916F915F914F913F912E
:105240002F910F900FBE0F901F9018951F920F92E5
:105250000FB60F9211242F933F934F935F936F9349
:105260007F938F939F93AF93BF93CF93DF93EF93EE
:10527000FF93C091E900CF708091EC00D82FD170DE
:1052800080FDD0E81092E9008091F000877F809344
:10529000F00078940E946A291092E9008091F00051
:1052A00088608093F000CD2BCF70C093E900FF9110
:1052B000EF91DF91CF91BF91AF919F918F917F91AE
:1052C0006F915F914F913F912F910F900FBE0F9073
:1052D0001F9018951F93CF93DF93CDB7DEB7AA9792
:1052E0000FB6F894DEBF0FBECDBFEBE7F4E08091C0
:1052F000F100819324E0E338F207C9F70E94D52436
:105300008091E80083FF2EC180917B0490917C0402
:10531000492F50E04A30510508F024C1FA01E55800
:10532000FF4F0C94302B803821F0823809F01AC1DD
:1053300008C08091770490917804992389F0826065
:105340000FC080917F048F70873008F00BC180936D
:10535000E9008091EB0085FB882780F91092E90035
:105360009091E800977F9093E8008093F10010926D
:10537000F100D1C0282F2D7F09F0F4C0882319F047
:10538000823061F0EFC080917D04813009F0EAC085
:10539000933009F080E0809378042EC080917D04E2
:1053A00081112AC080917F048F702FEF280F263043
:1053B00008F0D8C08093E9002091EB0020FF1CC0CA
:1053C000933021F48091EB00806214C09091EB0047
:1053D00090619093EB0021E030E0A90102C0440FFE
:1053E000551F8A95E2F74093EA001092EA008091F7
:1053F000EB0088608093EB001092E9008091E80058
:10540000877F8093E8000E948727ACC08111AAC0E3
:1054100010917D041F778091E3008078812B809329
:10542000E3008091E800877F8093E8000E9487274F
:105430008091E80080FFFCCF8091E300806880933A
:10544000E300111102C082E001C083E080937A047E
:1054500089C08058823008F085C080917D04909189
:105460007E048C3D53E0950779F583E08A838AE2D8
:1054700089834FB7F894DE01139620E03EE051E2B5
:10548000E32FF0E050935700E49120FF03C0E29532
:10549000EF703F5FEF708E2F90E0EA3010F0C7960C
:1054A00001C0C0968D939D932F5F243149F74FBF64
:1054B0008091E800877F8093E8006AE270E0CE0187
:1054C00001960E94932616C060917F04709180041B
:1054D000AE014F5F5F4F0E94D725BC01892B09F4B5
:1054E00041C09091E800977F9093E80089819A816C
:1054F0000E94F1268091E8008B778093E80032C00B
:10550000803881F58091E800877F8093E800809162
:1055100076048093F1008091E8008E7772CF81113C
:1055200021C080917D0490917E0499270297D4F444
:105530008091E800877F8093E80080917D048093CC
:1055400076040E94872780917604811106C080919D
:10555000E30087FD02C081E001C084E080937A040B
:105560000E94C1248091E80083FF0AC08091E80076
:10557000877F8093E8008091EB0080628093EB004E
:10558000AA960FB6F894DEBF0FBECDBFDF91CF91C4
:105590001F9108950895CF9380917A048823A1F0F4
:1055A000C091E900CF709091EC00892F817090FD3F
:1055B00080E8C82B1092E9008091E80083FD0E94EA
:1055C0006A29CF70C093E900CF910895AA1BBB1B35
:1055D00051E107C0AA1FBB1FA617B70710F0A61BF3
:1055E000B70B881F991F5A95A9F780959095BC0114
:1055F000CD01089597FB072E16F4009407D077FD90
:1056000009D00E94E62A07FC05D03EF490958195CA
:105610009F4F0895709561957F4F0895A1E21A2ECE
:10562000AA1BBB1BFD010DC0AA1FBB1FEE1FFF1F46
:10563000A217B307E407F50720F0A21BB30BE40B96
:10564000F50B661F771F881F991F1A9469F76095DD
:105650007095809590959B01AC01BD01CF01089597
:10566000EE0FFF1F0590F491E02D09948F929F9209
:10567000AF92BF92CF92DF92EF92FF92CF93DF93E0
:10568000EC01688179818A819B81611571058105B1
:10569000910521F464E279ED8BE597E02DE133EF9C
:1056A00041E050E00E94FA2B49015A019B01AC01F4
:1056B000A7EAB1E40E94192C6B017C01ACEEB4EFB7
:1056C000A50194010E94272CDC01CB018C0D9D1DAE
:1056D000AE1DBF1DB7FF03C00197A109B048888365
:1056E0009983AA83BB839F77DF91CF91FF90EF903F
:1056F000DF90CF90BF90AF909F908F9008950E94C1
:10570000362B089580E091E00E94362B0895A0E0AA
:10571000B0E08093000190930101A0930201B09347
:1057200003010895FB01DC0102C005900D92415078
:105730005040D8F70895FB01DC0104C08D91019021
:10574000801921F441505040C8F7881B990B0895E7
:10575000DC01CB01FC01F999FECF06C0F2BDE1BD31
:10576000F89A319600B40D9241505040B8F7089520
:10577000F999FECF92BD81BDF89A992780B5089519
:10578000A8E1B0E042E050E00C94AA2BDC01A40FA9
:10579000B51F4150504048F0CB01840F951F2E910A
:1057A0000E94D72B41505040D0F70895262FF999E9
:1057B000FECF92BD81BDF89A019700B4021639F070
:1057C0001FBA20BD0FB6F894FA9AF99A0FBE089541
:1057D0000396272F0E94D72B0E94D62B252F0E949D
:1057E000D72B242F0C94D72B0196272F0E94D72B31
:1057F0000C94D62B052E97FB1EF400940E94112CBE
:1058000057FD07D00E940E2B07FC03D04EF40C94DA
:10581000112C50954095309521953F4F4F4F5F4F3C
:10582000089590958095709561957F4F8F4F9F4F0C
:1058300008950E942C2CA59F900DB49F900DA49FBD
:10584000800D911D11240895B7FF0C94192C0E940E
:10585000192C821B930B0895A29FB001B39FC00126
:10586000A39F700D811D1124911DB29F700D811D8C
:0A5870001124911D0895F894FFCF54
:10587A0001000000FF0800FFFF0000FF7FFF00009B
:10588A00FF0000FF0000FF0000FF0160014001501F
:10589A000170037CC8007802232427249B249724C0
:1058AA009324262401E200E900EA00B500B600B715
:1058BA0000CD008301CC008A0192019401210223C8
:1058CA000224022502260227022A02B300B4006F2C
:1058DA00007000818283E200E900EA00B500B600A8
:1058EA00B700CD008301CC008A0192019401210204
:1058FA00230224022502260227022A02B300B40048
:10590A006F007000818283F5953132339392676616
:0C591A00363534979694F0F1F4F6F7005F
:00000001FF
